:020000040000FA
:1000000083160F3086001530850083121A308C005D
:10001000840000308E000E1016200E181C200E18C2
:1000200020200E1047200E184D200B28051E08001A
:10003000051A18280E14080006080F398D0008004C
:100040000C083F200E1044200E182C280C088400A9
:100050000D0880008C0A08000C088F008C0A1A30EA
:100060000F028F0303193A280F0884000008840A3E
:1000700080002F281A3084000D08800008004F30BF
:100080000C0203190B28080005190E140800051CA2
:100090000800051849280E140800000000001A3056
:1000A00084008F008F0A0008000EF03986000F08C8
:1000B0000C02031962280F088400000884038000E2
:0800C0008F0A57288C03080089
:02400E00F13F80
:00000001FF
